:1000000020C100003AC1000038C1000036C1000024
:1000100034C1000032C100000C94E9080C941909A5
:100020002CC100002AC1000028C1000026C1000028
:1000300024C1000022C1000020C100001EC1000038
:100040001CC100001AC1000018C1000016C1000048
:1000500014C1000012C1000010C100000EC1000058
:100060000C94160A0C94210A08C1000006C1000075
:1000700004C1000002C1000000C10000FEC0000079
:10008000FCC00000FAC00000F8C00000F6C000008C
:10009000F4C00000F2C00000F0C00000EEC000009C
:1000A000ECC00000EAC00000E8C00000E6C00000AC
:1000B000E4C00000E2C00000E0C00000DEC00000BC
:1000C000DCC00000DAC00000D8C00000D6C00000CC
:1000D000D4C00000D2C00000D0C00000CEC00000DC
:1000E000CCC00000CAC00000C8C00000C6C00000EC
:1000F000C4C00000C2C00000C0C00000BEC00000FC
:10010000BCC00000BAC00000B8C00000B6C000000B
:10011000B4C00000B2C00000B0C0000075C4000050
:10012000ACC00000AAC00000A8C00000A6C000002B
:10013000A4C00000A2C00000A0C000009EC000003B
:100140009CC000009AC0000098C000000C948B096D
:1001500094C0000092C0000090C000008EC000005B
:100160008CC000008AC0000088C0000086C000006B
:1001700084C0000082C0000080C000007EC000007B
:100180007CC000007AC0000078C0000076C000008B
:1001900074C0000072C0000070C000006EC000009B
:1001A0006CC000006AC0000068C0000066C00000AB
:1001B00064C0000062C0000060C000005EC00000BB
:1001C0005CC000005AC0000058C0000056C00000CB
:1001D00054C0000052C0000050C000004EC00000DB
:1001E0004CC000004AC0000048C0000046C00000EB
:1001F00044C000000C94F8130C94A614FD03FF03F4
:10020000010403040504070409040B041D041F046E
:100210002104230425042A0427042904ED0B130CCC
:100220003A0C630C6C0C710CB80CBD0CDC0CE30CC0
:10023000EB0C7D0C850C8D0C980C9A0C9C0CA40C72
:10024000AD0C11241FBECFEFCDBFDFE2DEBF10E249
:10025000A0E0B0E2EEE6FBE202C005900D92AA3902
:10026000B107D9F72BE2AAE9B0E201C01D92A03E86
:10027000B207E1F779D20C94B515C2CE84E0809331
:1002800056008CE189D3809363008BEB80936600EA
:1002900080E88093650081E08093600088ED84BFF2
:1002A0001092410083E08093500080915100833090
:1002B000E1F78091500081608093500088E1809345
:1002C00055008091510080FFFCCF809150008061EB
:1002D000809350008091510084FFFCCF88ED84BF53
:1002E00084E0809340000895E0E7F0E085818E7F10
:1002F0008583E0E0FAE08FEB9DE586A397A380EE8F
:100300009EE280A391A382E0808308958091200AD9
:100310009091210A813E2EE2920718F020918221CD
:1003200006C0803E2EE2920721F020917F2120938B
:100330006A0020910520222321F080910520815020
:1003400033C0885F9A42813D974080F110929A2095
:1003500080919B2090919C20A0919D20B0919E2007
:100360000196A11DB11D80939B2090939C20A0938A
:100370009D20B0939E2080919B2090919C20A091E5
:100380009D20B0919E20892F9A2FAB2FBB27809361
:10039000A22180919B2090919C20A0919D20B091C2
:1003A0009E208093A12186E08093052080910720E4
:1003B000909108200196B1F4809109208F3F91F02F
:1003C00080910620811106C0809106208150809383
:1003D00006200895809114019091150180930720C3
:1003E000909308200895009709F45EC00CF457C05C
:1003F00040E020916B0030E02093802130938121F8
:1004000020918021309181213695322F22273795F6
:100410002795209380213093812150916A0020916B
:10042000802130918121250F311D2093802130932F
:1004300081210000209180213091812128173907E6
:1004400028F410928021109281210895209180211A
:1004500030918121280F391F2115304238F08FEF5C
:100460009FE18093802190938121089520918021A4
:1004700030918121442329F0A901481B590BCA015D
:1004800002C0820F931F80938021909381218091DD
:100490008021909181218F7780936A0008959195B2
:1004A0008195910941E0A5CF0895CF93DF93C09145
:1004B000200AD091210A80910320909104209E016E
:1004C000281B390B209383213093842180919A201B
:1004D00081114BC080918321909184218E3C9F4F4C
:1004E000D4F480918321909184218B369F4F9CF08E
:1004F00080910220882321F080910220815008C041
:1005000080916A008093822181E080939A208CE020
:10051000809302202AC08CE0809302208091832166
:10052000909184218A369F4F1CF08FEF9FEF02C07D
:1005300081E090E080937D2190937E2180918321C2
:100540009091842120917D2130917E2160E370E0A3
:100550000E948C15261B370B20937D2130937E2122
:1005600080917D2190917E213EDF80919A20813083
:1005700029F58091832190918421C39794F08091F3
:100580000220882331F08091022081508093022044
:1005900015C080916A0080937F2183E080939A2028
:1005A0000DC08091832190918421873991051CF49D
:1005B00081E090E002C08FEF9FEF15DFC093032032
:1005C000D0930420DF91CF9108958617970779F093
:1005D0006817790728F49C01261B370BB90109C05D
:1005E0008617970718F4681B790B03C0089560E01D
:1005F00070E0CB010895CF93DF938091002090911C
:100600000120892B51F080910020909101200197C9
:10061000809300209093012043C080E490E0809379
:10062000002090930120809107209091082001964E
:10063000B9F1809114019091150120910920263083
:1006400018F467E771E002C06EEE72E00E94781560
:10065000EC0180910720909108208C179D0758F499
:100660006091072070910820CE01AFDF029718F04B
:1006700080EC9DE511C08091072090910820C8175B
:10068000D90770F46091072070910820CE019DDF9A
:10069000029730F08FEB9DE58093360A9093370AEE
:1006A000DF91CF910895AC01460F571F861B970B22
:1006B0002091200A3091210A24173507C8F720918C
:1006C000200A3091210A8217930790F70895E0E8F5
:1006D000F6E08FE0808385E0848308951F93CF93B5
:1006E000DF93C0E4D0E0198180E4898340E250E0E8
:1006F00068EB7BE280E290E00E94520F1983DF9169
:10070000CF911F9108951F93CF93DF93C0E4D0E062
:10071000198180E489838BEB95E20E94880F81E048
:100720000E949A0F1983DF91CF911F910895089528
:100730000F931F932091A4208EEE92E0289FA0019A
:10074000299F500D112444525A4D08E913E02EEE12
:1007500032E060E081E80E9435131F910F91089507
:100760001CBEEEEFF0E40994B9DF8091B82B88232A
:1007700069F080E2E8EBFBE2ABEBB5E201900D92B1
:100780008A95E1F71092BB25BEDFEADF87E0809310
:10079000A200789473DDCBDFAFD749D16CD160E094
:1007A00080E003D1EFD08CE0E3D073D517D630D6FC
:1007B0008EDF60E870E28EE891E20E94AE150000E4
:1007C0000000000000000000000000000000000029
:1007D0000000000000000000000080919F2088239E
:1007E00071F3E091BA238E2F90E088309105A0F448
:1007F000FC01E250FF4F0C949F1568D10DC0D8D179
:100800000BC064D209C0E8D207C073D305C0FBD3C4
:1008100003C0FAD301C06AD410929F20D0CF0895AC
:100820000895E09109208E2F90E08830910590F492
:10083000FC01EA5FFE4F0C949F15B9D10BC045D265
:1008400009C0C9D207C054D305C0DCD303C04DD4FE
:1008500001C0BED48091140180939721809115012D
:100860008093982180912401809399218091250182
:1008700080939A218091200A8093A3218091210A5C
:100880008093A421809114019091150186349140A8
:1008900080F08091140190911501893A914048F4BB
:1008A00080911401909115018093D82B9093D92BAE
:1008B00000008091A220882339F016DD1092A2203A
:1008C00081E08093A12008958091A120882341F0A8
:1008D00080919A20833019F419DD8DDE01C0E5DDA9
:1008E0008091A020882351F08091140190911501EE
:1008F0008093D82B9093D92B1092A0209091A42074
:1009000081E0911180E08093A42008950F931F93BC
:1009100081E08093A7208093A22008E913E02DE7CF
:1009200030E04CED55E260E081E80E94351381E053
:100930001F910F9108951092A720089581E00895C6
:1009400081E0089510922002982F9C7193689093F3
:10095000200287FF03C080E192E002C080E090E0C7
:10096000892B809321021092220210922602089570
:10097000E0E0F2E010AA836880AB80E181AB12AACC
:1009800016AA0895E0E0F2E010A683E880A78FE2BF
:1009900081A712A616A60895AAECB1E092E09C9356
:1009A000E82FF0E084911C920895909171009D7F52
:1009B0009093710010920002623011F09CE101C02E
:1009C0009EE19093010290E490930202811102C093
:1009D00080E401C080EC80930302613011F084E078
:1009E00001C083E08093040280E2D6DF80930C0292
:1009F00081E2D2DF80930D02109218021092190248
:100A000081E080930002BECF1F920F920FB60F922B
:100A100011248F93000000000000000081E080930B
:100A200023028F910F900FBE0F901F901895CF93B8
:100A3000DF93E0E7F0E082818B7F8283C0E2D3E046
:100A40008DE0888380E4898389E08A8383E3A4DF5F
:100A5000888782E3A1DF898787E39EDF8A8786E331
:100A60009BDF8B87E0E2F6E08081836080831482E5
:100A7000DF91CF910895E0E7F0E080818E7F808361
:100A800080E8809300010895E0E0F1E0108A80E4BE
:100A9000808B10A280A310AA80ABE0E4F1E010826A
:100AA00080831092A6201092A5201092A42010926C
:100AB0008C2110928D2110928A2110928B21089501
:100AC0008093BA2381E080939F200895CF93DF9392
:100AD00010920920D9DFC0E0D1E01EAA94E298ABC1
:100AE00019AA49E54AAB32E03BAB60910B2070910B
:100AF0000C206CAB7DAB6BEB73E268AF79AF1AAED9
:100B00008BE38CAF83E08DAF1EAE28A9206828ABA5
:100B100010924601E0E4F1E090831092410140938D
:100B200042018093430140910D2050910E2040934B
:100B30004401509345014AEA51E2409348015093E1
:100B4000490110924A0129E320934C0180934D0101
:100B500010924E01208120682083188A20E4288B7F
:100B600024E0288B898B85E98A8B80E18B8B47E792
:100B700051E04C8B5D8B988F398F1A8E8CED95E2FE
:100B80008C8F9D8F1E8E68EC70E084EF91E08BDD82
:100B900088EC90E0809307209093082081E0809378
:100BA000062088898068888BDF91CF910895089509
:100BB000EF92FF921F93CF93DF9311E010930920E0
:100BC00063DFC0E0D1E018AA80E488AB94E098AB82
:100BD00019AA1AAA6BE46BAB1CAA1DAA1EAA2AE0CA
:100BE00030E228AF39AF1AAEA0EAACAF58E05DAF43
:100BF0001EAE88A9806A88ABE0EAF8E085E58083CC
:100C0000808310924601E0E4F1E044E240831092D8
:100C1000410189E58093420132E030934301E09045
:100C20000B20F0900C20E0924401F09245018BEBF8
:100C3000E82E83E2F82EE0924801F09249011092EA
:100C40004A018BE380934C0183E080934D01109225
:100C50004E0120812068208398A389A325E92AA337
:100C60006BA367E771E06CA37DA3A8A759A71AA699
:100C7000EAECF8E2ECA7FDA71EA6988B898B2A8BDD
:100C800080E18B8B6C8B7D8B488F398F1A8E8CED2E
:100C900095E28C8F9D8F1E8E68EC70E084EF91E062
:100CA00002DD88EC90E08093072090930820109359
:100CB000062088A1806888A388898068888BDF9156
:100CC000CF911F91FF90EF90089508951F93CF93B8
:100CD000DF9312E010930920D7DEC0E0D1E01EAA16
:100CE00094E298AB19AA39E53AAB1BAB40910B20C3
:100CF00050910C204CAB5DAB4BEB53E248AF59AF7E
:100D00001AAE8BE38CAF83E08DAF1EAE28A92068AE
:100D100028AB10924601E0E4F1E09083109241018B
:100D2000309342018093430120910D2030910E2099
:100D300020934401309345012AEA31E2209348018F
:100D40003093490110924A0129E320934C0180938A
:100D50004D0110924E01208120682083188A20E4E2
:100D6000288B64E0688B898B55E95A8B40E14B8B6B
:100D700027E731E02C8B3D8B988F198F1A8EECED85
:100D8000F5E2EC8FFD8F1E8E68A389A35AA34BA3B7
:100D90002CA33DA384E388A719A71AA68AEC98E29E
:100DA0008CA79DA71EA668EC70E084EF91E07BDC29
:100DB00088EC90E0809307209093082081E0809356
:100DC000062088898068888B88A1806888A3DF9145
:100DD000CF911F91089508951F93CF93DF9313E050
:100DE0001093092051DEC0E0D1E010924601E0E40A
:100DF000F1E024E220831092410199E590934201B1
:100E000082E08093430140910B2050910C2040934D
:100E10004401509345014BEB53E2409348015093FA
:100E2000490110924A018BE380934C0110934D01CC
:100E300010924E018081806880831EAA28AB19AA77
:100E40009AAB1BAB80910D2090910E208CAB9DAB8B
:100E50008AEA91E288AF99AF1AAE89E38CAF1DAFF1
:100E60001EAE88A9806888AB18A250E458A344E05D
:100E700048A319A21AA23BE43BA31CA21DA21EA2D6
:100E80008AE090E288A799A71AA620EA2CA798E002
:100E90009DA71EA688A1806A88A385E58093A008E7
:100EA000188A588B488B198B85E98A8B3B8B47E7CF
:100EB00051E04C8B5D8B288F998F1A8E8CED95E2CB
:100EC0008C8F9D8F1E8E68EC70E084EF91E0EBDBE1
:100ED00088EC90E0809307209093082081E0809335
:100EE000062088898068888BDF91CF911F910895B3
:100EF00008951F93CF93DF9314E010930920C4DD6E
:100F0000C0E0D1E018AA80E488AB18AB19AA1AAAED
:100F10003BE43BAB1CAA1DAA1EAA8AE090E288AF64
:100F200099AF1AAE50EA5CAF88E08DAF1EAE98A9BB
:100F3000906A98AB95E59093A00810924601E0E482
:100F4000F1E094E290831092410199E5909342017F
:100F500092E09093430160910B2070910C2060937C
:100F60004401709345016BEB73E260934801709309
:100F7000490110924A019BE390934C0193E09093B6
:100F80004D0110924E01208120682083188B998B8F
:100F900045E94A8B3B8B27E731E02C8B3D8B588F03
:100FA000898F1A8E6CED75E26C8F7D8F1E8E18A363
:100FB00099A34AA39AE49BA32CA33DA393EC98A7DF
:100FC00089A71AA68AEC98E28CA79DA71EA668ECB2
:100FD00070E084EF91E067DB88EC90E0809307207D
:100FE0009093082081E08093062088898068888B10
:100FF00088A1806888A388898061888BDF91CF91E0
:101000001F9108950895FFCFCF93DF9386E08093DB
:1010100009203ADDC0E0D1E01EAA84E288AB19AA1B
:1010200039E53AAB93E09BAB40910D2050910E20F7
:101030004CAB5DAB4AEA51E248AF59AF1AAE29E377
:101040002CAF9DAF1EAE28A9206828AB1092460198
:10105000E0E4F1E08083109241013093420122E00C
:101060002093430140910B2050910C204093440168
:10107000509345014BEB53E2409348015093490193
:1010800010924A013BE330934C0190934D01109232
:101090004E01908190689083188A90E4988B888B99
:1010A000198A95E99A8B90E19B8B4CED55E04C8B1E
:1010B0005D8B888F298F1A8E8CED95E28C8F9D8F9A
:1010C0001E8E68EC70E084EF91E0EDDA80E991E04B
:1010D000809307209093082081E0809306208889E0
:1010E0008068888BDF91CF9108950895CF93DF9327
:1010F00087E080930920C8DCC0E0D1E01EAA84E22A
:1011000088AB19AA39E53AAB93E09BAB40910D202F
:1011100050910E204CAB5DAB4AEA51E248AF59AF5B
:101120001AAE29E32CAF9DAF1EAE28A9206828ABCC
:1011300010924601E0E4F1E0808310924101309387
:10114000420122E02093430140910B2050910C205A
:1011500040934401509345014BEB53E240934801C7
:101160005093490110924A013BE330934C01909314
:101170004D0110924E01908190689083188A90E4FE
:10118000988B95E2988B198A95E99A8B90E19B8BC5
:101190004CED55E04C8B5D8B888F298F1A8E8CED32
:1011A00095E28C8F9D8F1E8E68EC70E084EF91E04D
:1011B0007ADA80E991E0809307209093082081E01B
:1011C0008093062088898068888BDF91CF9108956D
:1011D00008951F920F920FB60F9211248F939F9331
:1011E00081E0809303011092100184E0809310014C
:1011F00087E791E080931401909315018091A420DA
:10120000811103C08EEE92E002C080E090E0845233
:101210009A4D80931C0190931D018091100180686C
:10122000809310019F918F910F900FBE0F901F9090
:1012300018951F920F920FB60F9211248F939F93C0
:1012400082E0809303011092200184E080932001CA
:1012500087E791E080932401909325018091A42059
:10126000811103C085E694E002C087E791E08452D3
:101270009A4D80932C0190932D01809120018068DC
:10128000809320019F918F910F900FBE0F901F9020
:101290001895E0E7F0E083818C7F838384818C7FE5
:1012A000848380818D7F8083E0E8F1E080EC82831D
:1012B000128688EC81831186A0E0B8E034E03C938C
:1012C00023E011962C93119714961C92149785ED98
:1012D00091E096968D939C93979716961C921697ED
:1012E000E0E4F8E030832183148286A397A316827A
:1012F000E0E6F6E0808180618083E0E4F9E083E16C
:101300008183148282E08683A6A3B7A310A611A6C8
:1013100081E0808308951F920F920FB60F921124DF
:101320002F933F934F935F938F939F93CF93DF932D
:101330001F92CDB7DEB78FEF80934C0980910920C3
:10134000873031F480912C02898390912D0202C064
:1013500090912C028091A320891B209168093091E3
:10136000690982308CF02A3F374070F42091680977
:101370003091690989301CF481E090E002C086E078
:1013800090E0820F931F18C020916809309169097D
:101390008F3FB4F42730310598F0209168093091DF
:1013A0006909883F1CF081E090E002C086E090E08F
:1013B000A901481B590BCA018093780990937909B8
:1013C0000F90DF91CF919F918F915F914F913F91BE
:1013D0002F910F900FBE0F901F901895E0E7F0E04F
:1013E00083818F7E8383E0E4F6E080818A6A808354
:1013F0008FEF848388E5828BE0EAF8E080E38383E3
:1014000084EC858387E08683178288E1848308954E
:10141000E0E7F0E08381877F8383E0ECF8E01182EE
:1014200088E58093550680E6808308951F920F9289
:101430000FB60F92112400000F900FBE0F901F9057
:1014400018951F920F920FB60F9211248F93EF935E
:10145000FF93E0EAF8E080818083FF91EF918F9124
:101460000F900FBE0F901F9018959FB7F894A0E5AE
:10147000B0E016968C911697897F16968C931697E6
:10148000E0E6F0E080E885838BEB868316968C910E
:101490001697846016968C938081816080839FBFAD
:1014A00008959FB7F894E82FF0E0E059FF4F60955A
:1014B0008081682360839FBF0895CF93863011F0A9
:1014C000C0E001C0C8E18091510081FD0DC09FB70F
:1014D000F894809150008260809350009FBF80916B
:1014E000510081FFFCCFC1DF6C2F636084E490E08A
:1014F000BED460E480E0CF91D4CF8091A82008953D
:101500008091A820813009F416CA0895F0D0FC011A
:1015100083818093A820811101C0F8C981E00895DA
:101520009091AA23892F807697FF07C0803491F489
:101530008091AB2381110EC003CA803459F480918D
:10154000AB23811107C08091B0239091B123892BE7
:1015500009F0F4C980E008958091AC238F770C9452
:10156000BF129091B020911102C080E00895E091E7
:10157000AD20F091AE200190F081E02D948189178B
:10158000A0F7E093AB20F093AC20228133812E0FA3
:101590003F1FE217F30798F49181943061F4928130
:1015A000891309C09381691306C0E093AB20F093BF
:1015B000AC2081E008959081E90FF11DEACFE0931E
:1015C000AB20F093AC20D1CFE091AD20F091AE20D4
:1015D0000190F081E02D228133812E0F3F1FFC010D
:1015E0004081E40FF11DE217F30748F48181843054
:1015F00031F0853039F08081E80FF11DF4CF80E0C3
:1016000090E00895CF0108951F93CF93DF93182F93
:10161000A8DF882339F1C091AB20D091AC20CE0156
:10162000D3DFEC01892B41F04C815D816B818A8194
:10163000B3D78111F4CF16C0E091AD20F091AE2068
:1016400092818381E92FF82FE10FF11DE10FF11D48
:101650000190F081E02D0190F081E02DDF91CF919C
:101660001F91099480E0DF91CF911F910895EF922F
:10167000FF921F93CF93DF93C82F60E072DF811139
:1016800002C010E02DC0E091AD20F091AE2092811B
:101690008381E92FF82FEC0FF11DEC0FF11DE08095
:1016A000F180D7011696ED91FC9117970995682F57
:1016B0008C2F57DF182F882321F3C091AB20D091B6
:1016C000AC20CE0181DFEC01892B21F08A810E94C0
:1016D000DF13F7CFD7011296ED91FC91139709957F
:1016E000812FDF91CF911F91FF90EF90089580910E
:1016F000AB209091AC200895E4C6CF938091B020A8
:10170000882311F0C0E008C01092B0201092B420DD
:101710001092B520CF910895E091AD20F091AE20C8
:101720000190F081E02D8481C81770F78C2F9FDF26
:10173000CF5FF2CFCF938091B0208823F1F0C0E04B
:10174000E091AD20F091AE20A081B18114968C91F2
:10175000C81798F492818381E92FF82FEC0FF11DBF
:10176000EC0FF11D0190F081E02D0084F185E02D5A
:10177000309709F00995CF5FE3CFCF9108950F938C
:101780001F93CF93DF931092B4231092B52310923E
:10179000B6231092B7231092B8231092B9238091E8
:1017A000AA2387FF07C02091B0233091B123232BB8
:1017B00009F457C38076803409F011C1E091AB235E
:1017C0008E2F90E0FC01E05AF109EB30F10508F0B2
:1017D00006C1E25FFE4F0C949F1581E08093A0202C
:1017E000809107209091082080939B218091072071
:1017F0009091082090939C218091822180939D213B
:1018000080917F2180939E2180916A0080939F2107
:1018100080916B008093A0216091B0237091B123DF
:101820008EE891E2D6C0109200088091AC2390918E
:10183000AD2380933608909337088091AE238F7044
:10184000809300086091B0237091B1238AEA91E2FD
:101850009CD68091B0239091B12320910D2030919E
:101860000E208217930709F4C7C280930D2090932E
:101870000E2026C0109240088091AC239091AD2399
:1018800080937608909377088091AE238F70809331
:1018900040086091B0237091B1238BEB93E275D631
:1018A0008091B0239091B12320910B2030910C2096
:1018B0008217930709F4A0C280930B2090930C2009
:1018C0008091092053C01092680910926909809193
:1018D000AC238093A32090C28091AC2380932406F4
:1018E0008BC2E091AC23F091AD23E830F10508F014
:1018F00076C0E75EFE4F0C949F1560E080E055D8FF
:101900008091AE231FD880E031C060E080E04DD8E8
:101910008091AE2317D881E029C061E081E045D8ED
:101920008091AE230FD88091AF2322D882E01EC0D1
:1019300083E01CC084E01AC060E080E036D880916B
:10194000AE2300D885E012C061E080E02ED88091FF
:10195000AE230E94A20486E009C062E080E025D8A0
:101960008091AE2380680E94A20487E0A9D844C277
:101970008091AC23809384063FC28091AC239091E8
:10198000AD23892B91F00E946E0380E2E8EBFBE22D
:10199000ABEBB5E201900D928A95E1F781E080937F
:1019A000BB250E9483030E946E03E9E7F0E091E00B
:1019B00088EDF89484BF90836091B0237091B12337
:1019C0008AE890E206C06091B0237091B12389E863
:1019D00090E2DBD511C20E94860481110DC2809174
:1019E000AA23982F907609F0C9C187FFFBC02091E8
:1019F000B0233091B1232115310509F4BFC18F7196
:101A000009F09EC08091AB23863071F0883009F4D4
:101A10008EC08111B3C12230310509F0AFC162E03F
:101A200070E084EB90E2D5CF8091AC239091AD2310
:101A3000292F332722303105A1F060F42130310500
:101A400009F09CC18091192090911A20DC016C91C1
:101A500070E05BC02330310589F12F30310509F189
:101A60008DC1E0911920F0911A202189821708F088
:101A700085C19927880F991F880F991FE0911B2016
:101A8000F0911C20E80FF91F80819181FC01628197
:101A900073817BD5E091B223F091B32382E08183FF
:101AA00035C080911D2090911E20009709F466C1D9
:101AB000DC0112966D917C91139727C09927813094
:101AC000910569F038F0029709F058C168E08AE69C
:101AD00090E208C064E070E08CE790E216C067E036
:101AE00083E790E2282FAAE5B0E2FC01819190E023
:101AF0008D939D938E2F821B8617C0F3660F6E5FAA
:101B00006093582070E088E590E23FD58091B02343
:101B10009091B1232091B4233091B523821793077C
:101B200008F06AC18093B4239093B52365C1213036
:101B3000310509F023C161E070E080EB90E249CF0C
:101B40008130C1F58091AB238A3009F017C1213073
:101B5000310509F013C18091B020882309F40EC12A
:101B6000C091AE23D091AF230091AD201091AE2053
:101B7000D801ED91FC918481C81708F0FFC060E0A6
:101B80008C2FEFDC882309F4F9C0DD27CC0FDD1F93
:101B9000F80182819381C80FD91FE881F9810680FD
:101BA000F781E02D09958093B22061E070E082EB2F
:101BB00090E20FCF823009F0E1C08091AB23811118
:101BC000DDC02230310509F0D9C08091AE232DD57A
:101BD00090E08093A9209093AA2062E070E089EAC7
:101BE00090E2F7CE8F7109F07DC08091AB238330F6
:101BF00009F4C4C018F48130A1F0C0C0853019F0D8
:101C0000893039F1BBC08091B0239091B123892BE9
:101C100009F0B4C08CEA9AE08093B6239093B7237E
:101C2000EBC08091B0239091B123892B09F0A6C01D
:101C30008091AC239091AD23019709F09FC08091D2
:101C4000B4209091B5208D7F8093B4209093B520DF
:101C5000D3C08091B0239091B123892B09F08EC01D
:101C600091D4882309F48AC02091AC233091AD230C
:101C70003327E0911920F0911A20818990E0821792
:101C8000930708F47BC039DD8091AC239091AD239C
:101C90008093B020882309F4AFC099278150904CDD
:101CA000880F991F880F991F20911B2030911C20AD
:101CB000820F931F8093AD209093AE20C0E0E091FF
:101CC000AD20F091AE200190F081E02D8481C81705
:101CD00008F092C060E08C2F97DC882309F44EC096
:101CE000CF5FEDCF8130E9F48091AB238B3009F0E9
:101CF00045C08091B0239091B123892B09F03EC05B
:101D00008091B020882309F439C0C091AE23D091CE
:101D1000AC238C2FACDC882389F16D2F8C2F74DCE5
:101D20002BC0823059F58091AB23813019F083307C
:101D300089F024C08091B0239091B123892BF1F4D4
:101D40008091AC239091AD23892BC1F48091AE2377
:101D500073D412C08091B0239091B123892B71F478
:101D60008091AC239091AD23892B41F48091AE23D7
:101D7000F6D48091AE232CD581113EC08091AA2348
:101D80008F718130D9F58091B020882309F469C022
:101D9000C091AE23D091AF230091AD201091AE2021
:101DA000D801ED91FC918481C81708F05AC060E019
:101DB0008C2FD7DB882311F1FE01FF27EE0FFF1FC9
:101DC000D80112968D919C911397E80FF91F00810D
:101DD0001181D8011696ED91FC9117970995682FFE
:101DE0008C2FBFDB882351F0D8011496ED91FC9124
:101DF00015970995882311F081E034C08091AA23BA
:101E00008F71823071F58091B020882351F1C0E04C
:101E1000E091AD20F091AE20A081B18114968C911B
:101E2000C817F8F492818381E92FF82FEC0FF11D88
:101E3000EC0FF11D00811181D8011696ED91FC91F6
:101E400017970995682F8C2F8CDB882351F0D801C8
:101E50001496ED91FC91159709958111CDCFCF5F27
:101E6000D7CF80E0DF91CF911F910F9108951BBED6
:101E7000FC0128ED24BF608308958091CF0187FD88
:101E8000FCCF08951F93CF93DF93C0ECD1E01A8568
:101E90008A8761E08BEC91E0EADF1A87DF91CF91CE
:101EA0001F910895CF92DF92EF92FF920F931F93AD
:101EB000CF93DF938C017B016A01DFDFCCECD1E0B3
:101EC000888188608883B801705FA601C7013DD60C
:101ED0008881877F8883DF91CF911F910F91FF9039
:101EE000EF90DF90CF900895CF93DF93C82FD62F38
:101EF000C4DFACECB1E08C9188608C93EC2FF0E007
:101F0000F05FD0838C91877F8C93DF91CF91089580
:101F10000F931F93CF938C01B0DFC0E0F801619164
:101F20008F018C2FE1DFCF5FC032C1F7CF911F91BE
:101F30000F910895CF93C82FA0DF20E2C29FC00168
:101F40001124E0ECF1E012829183808385E3CF914C
:101F500099CF4091CA01E62FF72F8093CA0184914F
:101F60004093CA010895E82FF0E0E652F44D8081D5
:101F70008F3F09F4FFCF9FB7F89480818F5F8083F4
:101F80009FBF0895E82FF0E0E652F44D8081811163
:101F900001C0FFCF9FB7F8948081815080839FBF9D
:101FA0000895CF93C82F80917C21C11105C088234B
:101FB00039F081E0E7DF04C0811102C081E0D3DFA6
:101FC000C0937C21CF910895282F2F70082E000CEC
:101FD000990B392F331F3327331F832F90E0820F44
:101FE000911D820F911D23E0880F991F2A95E1F71B
:101FF000885A9E4D08950F93E8ECF4E080818F7D20
:10200000808380818F7D8083E0E6F1E202E00593AA
:10201000109262211092632100E2069300E406937D
:10202000E8E5F1E200E2069300E40693EAEAF3E26F
:1020300014861586168617861286138610924D21F1
:102040000F9108950F9385E080934D21E1E6F1E231
:1020500004E00593E9E5F1E204E005930F910895AA
:102060000F9383E080934D2110926221109263219F
:10207000E0E6F1E202E006930F910895E091B623C5
:10208000F091B723309709F009940895282F2F7005
:10209000082E000C990B392F331F3327331F832F42
:1020A00090E0820F911D820F911D029749E0489F99
:1020B0009001499F300D1124C90189509F4D089509
:1020C000AF92BF92DF92EF92FF920F931F93CF9345
:1020D000DF93D82EDBDFEC018D2D76DF7C01DC0178
:1020E0001196EC91E770E150E73040F4F0E0EE0F2C
:1020F000FF1FE457FF4D0081118102C008E010E08E
:102100002D813E818B819C814881D7FE4AC0F70199
:1021100066817781260F371F2D833E832817390765
:10212000A1F1BC01621B730B9B01211574E0370701
:1021300038F02FEF33E0C901B801DAD4281B390B8E
:1021400041FF0AC0C901B801D3D4AC0191E0452BCD
:1021500009F090E0892F01C080E0988180FB91F91F
:102160009883D70116961D921C92179712962D935D
:102170003C93139729813A818D819E81820F931F11
:1021800014968D939C93159708C041FF78C04D7F9E
:1021900048831682178212821382F70102E00693A7
:1021A00085C0D7011296AD90BC90139742FF0FC027
:1021B000E981FA81B8019CD4B0E4DB9EB00111241E
:1021C00069587F4DAC01CF01820F931FBED42D8182
:1021D0003E812A0D3B1D2D833E838B819C8182177E
:1021E000930710F48D839E83F70126813781A21611
:1021F000B30609F044C02D813E818217930709F48C
:102200003EC0AC01421B530B9A01211554E0350727
:1022100050F02FEF33E0C901B8016AD4B901681B4F
:10222000790BCB0107C0C901B80162D4D901A81B41
:10223000B90BCD01F701128213828017910798F430
:10224000888184608883F0E4DF9EC001112489586E
:102250009F4DD70114968D939C93159716960D93C9
:102260001C9317979ACF49815A812D813E81240F63
:10227000351FF70124833583868397838ECF88812A
:1022800080FF14C08E7F8883EF81F885309771F0CE
:102290006D817E814D2D80E0DF91CF911F910F9157
:1022A000FF90EF90DF90BF90AF900994DF91CF91B6
:1022B0001F910F91FF90EF90DF90BF90AF90089526
:1022C0000F93CF93DF9380914D21833029F4D6DE95
:1022D000DF91CF910F918FCE2091492130914A21EA
:1022E000C091B423D091B523C21BD30B61F580916B
:1022F0004B2190914C21820F931F80934B219093FF
:102300004C212091B0233091B1238217930721F003
:102310008091B620882331F084E080934D21E8E558
:10232000F1E236C0E091B823F091B923309799F0EB
:102330000995882381F01092492110924A21C09179
:10234000B423D091B523C034D10528F01092B62023
:10235000C0E4D0E003C081E08093B620C093622146
:10236000D09363218091492190914A212091B223F9
:102370003091B323280F391F2093642130936521B6
:10238000C80FD91FC0934921D0934A21E0E6F1E25A
:1023900002E00693DF91CF910F9108950F93CF93B1
:1023A0008091CC0480FF63C021E02093CC0488E5B9
:1023B00091E2FC0100E80693E0E6F1E200E8069312
:1023C0002093CA04FC0100E1069380914D218823EB
:1023D00029F08350823008F451DE0DDE80915A21BD
:1023E00090915B21089709F044C088E0E9E0F1E2B0
:1023F000AAEAB3E201900D928A95E1F78091C804B0
:1024000080628093C8048091C80480628093C8046D
:10241000B6D9C82F811102C015DE2BC08091AA2326
:1024200087FF0DC010924B2110924C211092492130
:1024300010924A2182E080934D2142DF1BC080919F
:10244000B0239091B123892B11F40ADE13C01092AE
:102450004B2110924C211092492110924A2181E087
:1024600080934D21E8E5F1E202E0069303C0C0E06D
:1024700001C0C1E08C2FCF910F910895CF93CFB7BA
:10248000F89481E08EDDEAECF4E080E4808380E281
:102490008083E1ECF4E0808181608083A9ECB4E08A
:1024A0008C9182608C93E8ECF4E08081806480837E
:1024B0008C9181608C93808180688083CFBFCF9125
:1024C0000895CF931092600080E30E945D0A80918E
:1024D000C00480648093C00481E080936000CFB723
:1024E000F894109259211092612110926921109252
:1024F00071218091F7208E7F8093F72080910021B9
:102500008E7F809300216AE170E082E022DD8F3FC0
:1025100009F48FE18093FA046BE170E082E019DD49
:102520008F3F09F48FE18093FB048091C0048160A8
:102530008093C0048091C00480688093C00480911F
:10254000C00480618093C00488E591E28093C60452
:102550009093C7048091C00480628093C0048FEF81
:102560008093C5048091C80482608093C80410924F
:102570007C2185E0F8DC82DFCFBFCF910895809386
:10258000C30408958091C3040895EAEAF3E28087C2
:1025900091876287738708951F93CF93DF93162FD8
:1025A000EA0112DDFC018181807CD1F5612F63702D
:1025B000613019F020F080E803C080EC01C080E4B5
:1025C000C038D105E1F050F4C032D105A1F0C034DB
:1025D000D10599F06097C9F491E018C0C11592E057
:1025E000D90779F0CF3F93E0D90769F0C115D14001
:1025F00061F495E00BC092E009C093E007C094E05D
:1026000005C096E003C097E001C090E0118226E08B
:102610002083982B918381818062818381E001C036
:1026200080E0DF91CF911F910895CEDCFC01818184
:1026300082FB882780F90895CF93C82FC5DCFC0161
:10264000818182FF0FC081818B7F81838C2F1EDD72
:10265000FC01908190FF06C09E7F90830780F085EB
:10266000E02D099581E0CF910895AF92BF92CF926E
:10267000DF92EF92FF920F931F93CF93DF93D82EA9
:10268000C62E5A01790102DDEC018D2D9DDC9C01E5
:10269000DC0111968C911197807C09F454C011963D
:1026A0008C911197807C803C21F011968C9182FD59
:1026B0004AC09FB7F894888180FF02C09FBF43C083
:1026C000816088839FBFA982BA82EB82FC821D82CF
:1026D0001E820F83188791E0C11004C0E114F10439
:1026E00009F090E0888190FB81F98B7F8883D7FE89
:1026F00002C0F90122C0D90111968C911197807CFA
:10270000803CC1F41196EC91E770E150E73040F461
:10271000F0E0EE0FFF1FE457FF4D6081718102C0B2
:1027200068E070E0C701E4D1892B21F088818E7FB9
:10273000888309C0F90112821382168217828D2DB7
:10274000BFDC81E001C080E0DF91CF911F910F914C
:10275000FF90EF90DF90CF90BF90AF900895EF92F1
:10276000FF920F93CF93C82F2FDC7C018C2F8EDC30
:10277000DC01F70102E005939C9190FF1BC09E7F56
:102780009C931796ED91FC911897309799F0D7018B
:10279000C7FF05C016966D917C91179704C01296DD
:1027A0006D917C9113974C2F81E0CF910F91FF9009
:1027B000EF900994CF910F91FF90EF900895CF93F0
:1027C000C82FCDDF8C2F00DCFC011182CF91089542
:1027D0000F93CF93C82FF8DBFC0181818460818344
:1027E00001E006938C2FBBDF81E0CF910F9108951C
:1027F0001F920F920FB60F9211240F932F933F93B6
:102800004F935F936F937F938F939F93AF93BF93F8
:10281000EF93FF938091CB0487FF08C080E88093FB
:10282000CA040E949A0B0E9411047EC08091CB04BE
:1028300082FF18C084E08093CA048091602186FFE3
:1028400073C08091CC0481FD6FC0A8DD81116CC084
:1028500080914D21813011F403DC66C0843009F091
:1028600063C021C08091CB0481FF26C082E08093A9
:10287000CA048091582186FF57C08091CC0481FD05
:1028800053C08CDD811150C080914D21823041F4C4
:1028900084E080934D21E8E5F1E202E0069344C034
:1028A000833009F041C0E1E6F1E204E00593E9E597
:1028B000F1E204E0059338C08091CB0484FF1DC091
:1028C00080E18093CA040E947D0B1092C304109291
:1028D000592196E09093582183E4809359211092D6
:1028E0006121909360218093612189E091E280933E
:1028F0005C2190935D217FDB17C08091CB0486FF24
:1029000008C080E48093CA0480E04BDB0E940F047F
:102910000BC08091CB0485FF07C080E28093CA047E
:1029200081E03FDB0E941004FF91EF91BF91AF91D6
:102930009F918F917F916F915F914F913F912F91D7
:102940000F910F900FBE0F901F9018951F920F922E
:102950000FB60F9211240F931F932F933F934F9312
:102960005F936F937F938F939F93AF93BF93CF9317
:10297000DF93EF93FF938091CC0481FF1AC082E034
:102980008093CC048091C5048195880FE8E5F1E23D
:10299000E81BF109208131812855314283E03695C9
:1029A00027958A95E1F7822F869520FD06C0C0E025
:1029B00005C0F4DC882319F386C0C0E8C80F8C2F4B
:1029C00003DBFC01208125FF7EC000E20693C111DC
:1029D00074C080914D21843019F450DB0CDB73C03E
:1029E00000915A2110915B218091B4239091B523DD
:1029F000C0914921D0914A2198012C0F3D1F821787
:102A0000930718F48C010C1B1D0B8091B22390913D
:102A1000B323A80169E071E28C0F9D1F96D0C00F0F
:102A2000D11FC0934921D0934A210034110569F484
:102A300080914B2190914C218C0F9D1F2091B023B0
:102A40003091B1238217930788F0C093B423D093B9
:102A5000B523E091B823F091B923309729F0099577
:102A6000811102C0EFDA2FC0FBDA2DC08091B423B0
:102A70009091B523C817D907D9F4E091B823F09104
:102A8000B923309779F30995882361F320914B217D
:102A900030914C218091492190914A21820F931FBE
:102AA00080934B2190934C211092492110924A21FE
:102AB000E8E5F1E202E0069306C0C03811F400DC5C
:102AC00002C08C2FFDDAFF91EF91DF91CF91BF9182
:102AD000AF919F918F917F916F915F914F913F91B6
:102AE0002F911F910F910F900FBE0F901F9018956F
:102AF000AA1BBB1B51E107C0AA1FBB1FA617B70724
:102B000010F0A61BB70B881F991F5A95A9F780953F
:102B10009095BC01CD01089597FB072E16F4009403
:102B200006D077FD08D0E4DF07FC05D03EF4909591
:102B300081959F4F0895709561957F4F0895EE0F91
:102B4000FF1F0590F491E02D0994FB01DC0102C008
:102B500001900D9241505040D8F70895FB01DC01DF
:0E2B600001900D920020E1F70895F894FFCF48
:102B6E0040000CE02E0AFFFFFFFF5580008000861C
:102B7E000A800A900A7D0A000044201F20000028C7
:102B8E002023200F200000000902190001010080FF
:102B9E00FA0904000001FFFFFF0007058101FF0392
:102BAE00010000001201000200000040EB0394BA85
:102BBE0000020102000100000003000000000000FE
:102BCE00000000000000000000004C6162726164B1
:102BDE006F72004573706F54656B00000403090437
:102BEE006465627567313233000206001000200002
:0A2BFE004000800000010002FF0308
:00000001FF
